:020000040000FA
:040000006B303A28FF
:08000800A000030EA100831209
:100010008B1C32288B1031181428B11C3228643004
:10002000010203183128182800001628172818285C
:1000300019281A281B281C281D281E281F283110A3
:10004000B114A810031005190314AA0DA90DA80DC9
:10005000B00B322831152A08AF002908AE00280855
:10006000AD00B11081010B11210E8300A00E200EF6
:02007000090085
:0C007400203084008001840A6030040207
:10008000031C3C281230B0009C218316FF239000F3
:10009000831283160C308505870183128501870141
:1000A000073099000030831691008312C830831600
:1000B0008100831231309000003083168C0083124F
:1000C00010308B00831600309B001C141A0883121A
:1000D000BC00831610309B001C141A088312BD004C
:1000E000E02181018E018F010B118B100B108C010F
:1000F0008B17882031199E20B30B86280310851991
:100100000314B90DF030390203192321F92179289C
:100110006400311808000B1D08000B11B1103114D8
:100120001230B000051D9928321483160113831272
:1001300008003210831601178312080031110130B4
:10014000B7008B132030370783169B001C141A0846
:100150008312A400A500C030A5061030370783160F
:100160009B001C141A088312A30000303707831663
:100170009B001C141A088312A2008B17321CC6287D
:1001800022090339A200A309A409A50922082D0206
:10019000031D1D2923082E02031D1D2924082F02DB
:1001A000031DF52801303702031DD9283D143E14E4
:1001B000A92102303702031DE028BD143E14AD21F1
:1001C00003303702031DE7283D153E14B1210430EA
:1001D0003702031DEE28BD153E14B5210530370248
:1001E000031DF5283D163E14B92125082F02031DD5
:1001F0001D2901303702031D00293D103E14BD2189
:1002000002303702031D0729BD103E14C1210330FF
:100210003702031D0E293D113E14C521043037025B
:10022000031D1529BD113E14C92105303702031DD8
:100230001C293D123E14CD211D29B70A0630370274
:1002400003180800A1280130B600B300B400B500BF
:10025000B70085018701B1138820B30B4F29031024
:1002600085190314B90DF030390203197629B40B3E
:100270004F29013037020319D12102303702031907
:10028000D421033037020319D72104303702031970
:10029000DA21053037020319DD219630B400311D13
:1002A0002C293111321C59292D090339AD00AE0911
:1002B000AF092F1CB1132F1C2C29B11B2C292E1870
:1002C0002C29B1178B1320303707BB002F08BA0039
:1002D000892110303707BB002E08BA008921003071
:1002E0003707BB002D08BA0089218B1785018701CC
:1002F000B70AB60106303702031C2C29E02108009A
:100300003E1C08003E101030BB003D08BA00892199
:1003100008008B133A0883161C159A003B089B00B3
:1003200055309D00AA309D009C1464009C189529AE
:100330001C1183128B170800FF30D000D415D5157F
:10034000D615D715D815D915DA15DB15DC15DD1539
:100350000800D2104E14CE100800D2114E15CE1146
:100360000800D2124E16CE120800D2134E17CE132A
:100370000800D3104F14CF1008005210CE144E10A6
:1003800008005211CE154E1108005212CE164E1210
:1003900008005213CE174E1308005310CF144F10FD
:1003A0000800303085060800033085060800063056
:1003B00087060800213087060800183087060800E5
:1003C0003D184E143D1CCE14BD184E15BD1CCE1547
:1003D0003D194E163D1DCE16BD194E17BD1DCE172B
:1003E0003D1A4F143D1ECF144E08D200CF00D3004B
:1003F00008008F08031908008F01D00F3B2BD00A8B
:10040000521C112A541D072AD40154161F2AD41D28
:100410000C2AD40154161F2A541E1F2AD401D414A6
:100420001F2AD41C162AD40154151F2A541D1B2A16
:10043000D401D4151F2A541E1F2AD4015415D21CCE
:10044000302A551D262AD50155163E2AD51D2B2AA0
:10045000D50155163E2A551E3E2AD501D5143E2AF1
:10046000D51C352AD50155153E2A551D3A2AD501E8
:10047000D5153E2A551E3E2AD5015515521D4F2A27
:10048000561D452AD60156165D2AD61D4A2AD60182
:1004900056165D2A561E5D2AD601D6145D2AD61C34
:1004A000542AD60156155D2A561D592AD601D6154D
:1004B0005D2A561E5D2AD6015615D21D6E2A571D7D
:1004C000642AD70157167C2AD71D692AD7015716E7
:1004D0007C2A571E7C2AD701D7147C2AD71C732A62
:1004E000D70157157C2A571D782AD701D7157C2AA2
:1004F000571E7C2AD7015715521E8D2A581D832A54
:10050000D80158169B2AD81D882AD80158169B2A2C
:10051000581E9B2AD801D8149B2AD81C922AD8018D
:1005200058159B2A581D972AD801D8159B2A581E62
:100530009B2AD8015815D21EAC2A591DA22AD901CE
:100540005916BA2AD91DA72AD9015916BA2A591EED
:10055000BA2AD901D914BA2AD91CB12AD9015915F4
:10056000BA2A591DB62AD901D915BA2A591EBA2A4A
:10057000D9015915521FCB2A5A1DC12ADA015A1620
:10058000D92ADA1DC62ADA015A16D92A5A1ED92AB8
:10059000DA01DA14D92ADA1CD02ADA015A15D92A52
:1005A0005A1DD52ADA01DA15D92A5A1ED92ADA01B2
:1005B0005A15D21FEA2A5B1DE02ADB015B16F82AD6
:1005C000DB1DE52ADB015B16F82A5B1EF82ADB013E
:1005D000DB14F82ADB1CEF2ADB015B15F82A5B1D14
:1005E000F42ADB01DB15F82A5B1EF82ADB015B1518
:1005F000531C092B5C1DFF2ADC015C16172BDC1D2C
:10060000042BDC015C16172B5C1E172BDC01DC14A1
:10061000172BDC1C0E2BDC015C15172B5C1D132B20
:10062000DC01DC15172B5C1E172BDC015C15D31CC1
:10063000282B5D1D1E2BDD015D16362BDD1D232BAA
:10064000DD015D16362B5D1E362BDD01DD14362BEC
:10065000DD1C2D2BDD015D15362B5D1D322BDD01E3
:10066000DD15362B5D1E362BDD015D1580214E0814
:10067000D2004F08D3005008D1000C305405031DA0
:1006800005120C305505031D85120C305605031D4F
:1006900005100C305705031D85100C305805031D3F
:1006A00087100C305905031D07110C305A05031D26
:1006B00007100C305B05031D87120C305C05031D11
:1006C00007120C305D05031D871151080E02031837
:1006D000952B12305405031D051612305505031DC8
:1006E000851612305605031D051412305705031DDB
:1006F000851412305805031D871412305905031D47
:10070000071512305A05031D071412305B05031D2F
:10071000871612305C05031D071612305D05031D98
:100720008715FF305002031908008F08031D0800C9
:10073000882051080E02031C952B18305405031D08
:10074000051206305405031D051618305505031D06
:10075000851206305505031D851618305605031DF4
:10076000051006305605031D051418305705031DE6
:10077000851006305705031D851418305805031DD4
:10078000871006305805031D871418305905031DBE
:10079000071106305905031D071518305A05031DAA
:1007A000071006305A05031D071418305B05031D9A
:1007B000871206305B05031D871618305C05031D84
:1007C000071206305C05031D071618305D05031D72
:0C07D000871106305D05031D8715080029
:084000000200030002000600AB
:02400E00CC01E3
:10420000010003000300030003000200020002009B
:1042100002000000000000000000FF00FF00FF009F
:10422000000000000000000000000000000000008E
:104230000000C000C000C000C000FF00FF00FF0081
:104240000100C300F300CF00FF00C300F300CF0064
:10425000FF00C300F300CF00FF00FF00FF00FF00DE
:10426000FF00FF00FF00FF00FF00FF00FF00FF0056
:10427000FF00FF00FF00FF00FF00FF00FF00FF0046
:10428000FF00FF00FF00FF00FF00FF00FF00FF0036
:10429000FF00FF00FF00FF00FF00FF00FF00FF0026
:1042A000FF00FF00FF00FF00FF00FF00FF00FF0016
:1042B000FF00FF00FF00FF00FF00FF00FF00FF0006
:1042C000FF00FF00FF00FF00FF00FF00FF00FF00F6
:1042D000FF00FF00FF00FF00FF00FF00FF00FF00E6
:1042E000FF00FF00FF00FF00FF00FF00FF00FF00D6
:1042F000FF00FF00FF00FF00FF00FF00FF00AA001B
:00000001FF
